:030000000219FDE5
:03000B000200A848
:03002B000201854A
:03005B0002033964
:030073000203265F
:1000800002030406080C10182030406080040608A3
:100090000C10182030406080A0C00003070F1F051F
:1000A000050D050305030302C2AF306308C2638573
:1000B000798AD2AF32C0D0C0E0206221E525601637
:1000C000E473E525F4C3334009758A00D263F579FA
:1000D00001D4F58AD262D0E0D0D0D2AF32C3E526C7
:1000E000334009758A00D263F57901EEF58AC26260
:1000F000E526F4602F30682520720DD0E0D0D0C204
:1001000092C296C294D2AF32C292C296C294206F6B
:100110000C206609740ED5E0FDE57B4290D0E0D05E
:10012000D0D2AF32758A00D263757900C28DD262A7
:10013000211D01C2306805206602D29201C23068DA
:1001400005206602D29401C2306805206602D2966C
:1001500001C2C29330680A2066077410D5E0FDD250
:100160009201C2C29530680A2066077410D5E0FD7E
:10017000D29401C2C29730680A2066077410D5E095
:10018000FDD29601C2C2AFC2AD53E6EFC0D0C0E00F
:10019000D2D3D2AFE57A6009E57760057577004183
:1001A000D3757701C2CEE52A6007207449152A214C
:1001B000F67800790020742EE580307E01F430E579
:1001C0000278FF53DACF207E0343DA20307E0343E8
:1001D000DA10C2D8C271E580307E01F430E50279D0
:1001E000FFC3E89970CB306103752A18207403753A
:1001F0002A18885CD27020740DE52B6004152B4101
:100200000643DA01C2D82070024179A85C2061025D
:10021000C270207431C3E894F0400374F0F8E8C46D
:10022000540F28F87984B703024146C313C31387D8
:1002300021200802C313200A06C3C898F8414628A3
:10024000F8500374FFF8C3E895655003E565F88836
:1002500022E52D54066022206B1FE536C333C333DD
:10026000F8E564C313C313F9C3952240028922E859
:100270002522F52250037522FF852224A824C3E5F8
:100280002495614002A8618825E566700241BDC3DE
:10029000E8AA669A5003E8FAE4F9EAC333FBE56892
:1002A000F45B29400D2567F8E56760021567400B90
:1002B00041BD0AC3E5679A5002056778FF8826C2E8
:1002C0006FC3E52694F84002D26FC3E52594404001
:1002D00002D26420CF0AD0E0D0D043E610D2AD32B3
:1002E000C2CF053AE57A6009E57860057578006166
:1002F0001C7578017801E52A6005307402152AC35F
:10030000E55C94014005755F00611C7560007569CE
:1003100000E55F2401F55F5003755FFFD0E0D0D0AA
:1003200043E610D2AD32C2AF53E67F7592FA7593B1
:10033000FFC260759104D2AF32C2AF53E6EFC2ADD7
:10034000C0D0C0E0C0F0D2D3D2AFA8FBA9FCE57A00
:100350006007C3E913F9E813F8C2D830710261AB42
:1003600053DACF207E0343DA10307E0343DA20D203
:1003700071E580307E01F420E502618288278928BA
:10038000A1D853DACF207E0343DA20307E0343DA4C
:1003900010C2D8C271307402A1C47800E580307EEA
:1003A00001F430E502A1C4885CA1AC53DACF207E11
:1003B0000343DA20307E0343DA10C27120610281E8
:1003C0008453DACF207E0343DA10307E0343DA20F1
:1003D000C2D8D27188578958C3E89555F8E995561F
:1003E000F97B007E087A00C3E8948CE994005005FC
:1003F000755B008176882178A2E6A8216055C3E864
:1004000094C8E994005008E4D2E4FB7A0A8151C30D
:10041000E89468E994015008E4D2E3FB7A0F815133
:10042000C3E894D0E994025008E4D2E2FB7A1E813A
:1004300051C3E894A0E994055008E4D2E1FB7A3C6A
:100440008151C3E89498E994085008E4D2E0FB7A1B
:10045000787E00C3E89559FCE9955AFD30E70AEC2F
:10046000F42401FCEDF43400FD755B00C3EC9AED5F
:0D0470009E5003755B018859895A855755C8
:10047D008558567802A1ACC3E89527F8E99528F977
:10048D00307C02A190307B02A190307A02A18920AC
:10049D00750281A7E9FDE8FC81C6E9C313F9E813EC
:1004AD00F8307902A189E9C313F9E813F83078021D
:1004BD00A189E9C313FDE813FC20612CC3EC941C46
:1004CD00ED9402400281DDED701EC3EC94C850180E
:1004DD000529E52970021529C3E529940A5002A1C1
:1004ED00C4755C00D270A1C4E52960021529788815
:1004FD00E6F97400207F087896B90302789EE62409
:10050D00FAFEE43400FFC3EC9EFCED9FFD9208B9AA
:10051D000310A2085007207609D276A12F3076025B
:10052D00C276A2085016B9030DECF42401FCEDF4CB
:10053D003400FD02054978007900A190B90315EC4E
:10054D0033FCED33FDC3EC940AFCED9400FD500437
:10055D007C007D00C3EC94FFED9400400678FF799C
:10056D0000A190EC8572F0A4C5F0A2F733F87900E4
:10057D0040030205AC78FF79000205ACE9C313F91D
:10058D00E813F8307C0EE9600278FFC3E81338F801
:10059D00E43400F9C3E894FFE99400400278FF8841
:1005AD005CD270206102A1C4741FF4552F4BF52F3E
:1005BD00C274EB7002D274752A18307403752A0A4E
:1005CD00306102A1D820740353DAFE207403752B19
:1005DD0006D0F0D0E0D0D0D2AD43E6103279010292
:1005ED0006087903020608790A020608791E020632
:1005FD0008796402060879C80206087817E4D5E080
:10060D00FDD8FAD9F6227A147B7802062F7A107B60
:10061D008C02062F7A0D7BB402062F7A0B7BC80253
:10062D00062F7902E4C295D5E0FDD294D5E0FDC246
:10063D0094D5E0FDD295D5E0FDE920E002D29230CF
:10064D00E002D296E573D5E0FDE920E002C29230DA
:10065D00E002C2967496D5E0FDD9C9EAF8D5E0FD61
:10066D00D8FBDBBEC29522C37C007D0075F0000572
:10067D00F0EA33FAEB33FB50F6EB13FBEA13FAC354
:10068D00E9FFE8FEE89AF8E99BF95004EFF9EEF876
:10069D00B3EC33FCED33FDD5F0DFEDF9ECF822E8EA
:1006AD0089F08A20D2D4F8A9F07B0030F70B7BFFBC
:1006BD00F42401F8E9F43400F9E88520F0A4ADF054
:1006CD00F8E98520F0A4AFF0FEED2EF974003FFAA5
:1006DD007C04C3EA13FAE913F9E813F8DCF48BF0A0
:1006ED0030F70AE8F42401F8E9F43400F9E889F068
:1006FD00C2D4F8A9F02222C3E54113F9E54013F85D
:10070D00C3E54498F8E54599F9500CC3E89480E9A0
:10071D0094FF401602073BC3E8947FE99400500311
:10072D0002073B787F790002073B788079FF884983
:10073D00894A22E5492546F8E54A3547F9854A2093
:10074D00E4300701F43548FA30E709C3EA94F04084
:10075D0015020779C3EA940F500302077978FF79E0
:10076D00FF7A0F020779780079007AF0C3E52495B6
:10077D0061500AC374019524500B020797E54A2076
:10078D00E70E020797E54A30E706884689478A480B
:10079D002278A5E6FAC3E54933F8E54A33F9D1AC39
:1007AD00E930E70BC3E89480E994FF4013E1D1C32E
:1007BD00E8947FE994005002E1D1787F7900E1D18E
:1007CD00788079FFE820E715C3E52398F84009C341
:1007DD00E8940140030207F878010207F8E8F424D1
:1007ED00012523F840030207F878FF884B2278A6ED
:1007FD00E6FAA847A9481206ACE930E70CC3E8941D
:10080D0001E994FF401602082DC3E894FFE9940016
:10081D00500302082D78FF790002082D780179FF29
:10082D00E920E715C3E54B98F84009C3E89401406A
:10083D00030208547801020854E8F42401254BF80A
:10084D00400302085478FF88242278FFC26420698F
:10085D003D206A12D264C3E541940A4009C3E525DF
:0F086D0094405002C26479A1E76023E541601F07
:10087C0074FF8541F0848539F0306A0375F005A466
:10088C00F8C5F0600278FFC3E895645002A864884C
:10089C006322C3E54094C8E5419400E5635003141A
:1008AC0001AF046002F563220208B72275E89022BA
:1008BC007883E6FFE5E820ECF7A8BDA9BE0570C378
:1008CC00E57094084052757000E9FA79A0E760442D
:1008DC00EA7007E571601B0208F2C3E895716010BD
:1008EC00E5715006600C140208FE0460F90208FE63
:1008FC00E571F571C39472401B7561C0C3940440DB
:10090C0013756180C39404400B756140C39404401B
:10091C000375610075BB0822E561F460020561E5B1
:10092C0070B4070375BB1022743279A787F0A4C585
:10093C00F0A2F733F8C3E895614002A861882288D9
:10094C0024882588268864227540007541F022C2CF
:10095C00AF75C820A8CCA9CDAA3A30CF010A75C86A
:10096C0024D2AFC3EA13FAE913F9E813F8AB3BACA2
:10097C003C883B893CC3E89BF8E99C20690A547F7E
:10098C00F9306702417521D2AD3D8A3DF9EA9D549B
:10099C007FFA600478FF79FFAE3EAF3F8B3E8C3F11
:1009AC00A83BA93CC3E89EF8E99FF9C3E54113FBBA
:1009BC00E54013FAE82AF540E93BF541500675404D
:1009CC00FF7541FF411CAA40AB41AC40AD417E04D8
:1009DC007F02C3EB940440021E1FC3EB9408400239
:1009EC001E1FC3ED13FDEC13FCDEF7C3EA9CFAEB00
:1009FC009DFBEF6009C3E913F9E813F8DFF7EA2868
:100A0C00FAEB39FB8A408B4150067BFF8B408B41C4
:100A1C00C3EB94025002D2673069047F03414778DC
:100A2C0092E6FFC3E537948240110FC3E53794A0DB
:100A3C0040010FC3EF940640027F057E02E541C4DE
:100A4C00540FF9E541C454F0F8E540C4540F28F8AC
:100A5C00C3E89EFAE99400FB4009C3EA9402EB94C4
:100A6C000050047A02E4FB41C1AA40AB41EBC4FE46
:100A7C00EAC4540F4EFCC3EA9CFAEB9400FBC3E8A7
:100A8C0013C313F8EA28FAEB3400FB8A408B41C3FA
:100A9C00EB94024002C2677802EBC4FE7B00EAC40E
:100AAC00540F4EFAC3EA98FA4005C3940250027AE6
:100ABC00027892E6FF30600241C1855192855293D3
:100ACC00D26043E680C3E49AF8E49BF9C3E833F8B8
:100ADC00E933F93067026154E8FAE9FBD3E913FD15
:100AEC00E813FC88518952C3EF94036038EF20E07F
:100AFC000DE82CF8E93DF9ECFAEDFB020B1DE828AA
:100B0C00F8E939F9C3E82402F8E93400F97AFE7BF4
:100B1C00FFC3EF9403400E8A538B54884D894E8C3F
:100B2C004F8D506188885389548A4D8B4E8C4F8DD4
:100B3C00503069127553F07554FF754FF07550FFB6
:100B4C007551F07552FF6188E8FAD3E813FC8851AF
:100B5C00C3EF94036020EF20E007E82CF8ECFA6177
:100B6C0074E8282402F87AFEC3EF940340088A53F1
:100B7C00884D8C4F618888538A4D8C4FE568C33300
:100B8C005002646BF5683060026192753402D26079
:100B9C0043E680E52D5406602DA840A941C3E91316
:100BAC00F9E813F8306904E92440F9C2AF53E67F41
:100BBC00759100C3E498F594E499F595759104D278
:100BCC006043E680D2AF22D26575430075200030B9
:100BDC006C03752040020BF2D26575430075204002
:100BEC00306C0375200078017901206720E52D54C5
:100BFC00066002C2657914E541C313700104F8C3A1
:100C0C00941440027814306904781B791BC3E833C0
:100C1C00F8C3E933F9206010E543600C306903D563
:100C2C003404D26D81AA719A0543E59BF45440B506
:100C3C002002819430690908C3E899400118812188
:100C4C0020650A08C3E899400261F28121C265C29D
:100C5C00AF53E67F7591003067127594007595FC63
:0E0C6C00759104D26043E680D2AF61F2AE40D3
:100C7A00AF41C3EE33FEEF33FF50047EFF7FFFC365
:100C8A00E49EF594E49FF595816CC3E53394015095
:100C9A000261F230650261F2D80281A88121C26D37
:100CAA00C2AF53E67F75910085539485549575912B
:100CBA0004854D92854E93D26043E680D2AFE52DEE
:100CCA0054066008206A020533020CE6306D0D20D6
:100CDA006C0A206507158115810215A32278003058
:100CEA0064053065027801E53775F007A4F9E5F087
:100CFA0028F5F0E9A2F013A2F113A2F213F537C313
:100D0A0094785003753778C3E53795384008D2662A
:100D1A00C292C296C294306002A120854F92855039
:100D2A0093D26043E68022207D16C2AF754202C28A
:100D3A0095D293306202D296D2AF759F40020F20AD
:100D4A00C2AF754202C295D297306202D292D2AF36
:100D5A00759F40020F20307243207D20C2AF75423A
:100D6A0003900163757B20C296C297306204D294C5
:100D7A00A17ED295D2AF759F41020F20C2AF7542B4
:100D8A0003900163757B20C292C293306204D294AD
:100D9A00A19ED295D2AF759F43020F20207D17C224
:100DAA00AF75420390013EC296306202D294D2AF2E
:100DBA00759F41020F20C2AF75420390013EC29255
:100DCA00306202D294D2AF759F43020F20207D1663
:100DDA00C2AF754204C293D297306202D294D2AFA4
:100DEA00759F43020F20C2AF754204C297D2933057
:100DFA006202D294D2AF759F41020F203072432013
:100E0A007D20C2AF754205900152757B08C294C21B
:100E1A0095306204D292C124D293D2AF759F400218
:100E2A000F20C2AF754205900174757B80C294C2CF
:100E3A0095306204D296C144D297D2AF759F4002D0
:100E4A000F20207D17C2AF754205900134C294303D
:100E5A006202D292D2AF759F40020F20C2AF754292
:100E6A0005900148C2943062EBD296D2AF759F408A
:100E7A00020F20207D16C2AF754206C297D2953066
:100E8A006202D292D2AF759F41020F20C2AF754261
:100E9A0006C293D295306202D296D2AF759F4302B0
:100EAA000F20307243207D20C2AF75420190017439
:100EBA00757B80C292C293306204D296C1CAD2971D
:100ECA00D2AF759F43020F20C2AF75420190015203
:100EDA00757B08C296C297306204D292C1EAD29355
:100EEA00D2AF759F41020F20207D17C2AF75420114
:100EFA00900148C292306202D296D2AF759F4302E5
:100F0A000F20C2AF754201900134C296306202D2FC
:100F1A0092D2AF759F41C26622900132757B00C2A0
:100F2A0092C296C294C293C297C295C26222788034
:100F3A0076FF0876FF0876FF0876FF0876030876BC
:100F4A000408760A087603087601087601788C7612
:100F5A00010876FF0876FF0876FF0876FF0876FF15
:100F6A000876030876FF0876FF0876FF08762508D4
:100F7A0076D00876FA0876FA0876040876FF0876B4
:100F8A000108760008767A0876FF08760108760165
:100F9A00087600087603087600227887E6FFC27290
:100FAA00BF0302D2727888E6C394036008C27DE662
:100FBA0030E102D27DC27E7889E630E102D27EC378
:100FCA00EF94026008758E01D273020FDC758E00F1
:100FDA00C273227880E6149000809378A5F678810F
:100FEA00E6149000809378A6F67886E61490008D31
:100FFA009378A7F67886E6F539C3940250037539D3
:10100A0002789CE67538FFB402037538A0B403036E
:10101A0075388278A3E61490009A93F566120F2326
:10102A0022227896E6FA7897E6FB7888E6B40305F2
:10103A00C3EB940EFB307F047A007BFFC3EB9AFC70
:10104A00C3948250027C827572000572EC8572F03C
:10105A00A4C3E5F0947D40F222D27F112C1205F947
:0F106A007A007B007C101205EFE55C2AFA740017
:101079003BFBDCF37C04C3EB13FBEA13FADCF7FE5E
:10108900C27F112C22E5EF20E60375200005209090
:101099003FFFE520146006901FFF14600093046071
:1010A9000375EF1253D9BF7581C043FF801205EA5A
:1010B90075EF0243B203E5B3240220E70DF521E5FC
:1010C900E320E0068521B343E301120F237580FF76
:1010D90075A40075F13075D4DF75900375A5FC759D
:1010E900F2FC75D50175A60175E241C292C296C29C
:1010F900941205FED293D297D2951205EAC293C2F1
:1011090097C295120F23E4F8F6D8FD756801120FFE
:10111900381215FD78988673753001C2AF1206032F
:101129001206131205F912061A1205F912062112EE
:1011390005F91217161206031206031205FEC2AFAD
:1011490078FA79FA308507D9FBD8F7021C00120F13
:10115900A4120FDD112B112C78988673120F2375A9
:10116900A90075B680757A0075881075890275C8E9
:101179002475910475D84075A82275B80275E69052
:10118900759B80759D0075D10E75BCC075BB0875C2
:10119900BA1175E8801205EAD2AF1208B4753600A3
:1011A90053DACF207E0343DA20307E0343DA10433B
:1011B900DA01C2D8C271120603D2617B037A0CE547
:1011C9005B70077A0CDB030211471205F9207003E3
:1011D900021147C270E55CC3940240E1E52F541F38
:1011E900855E5DF55EB55DD5DAD5C26153DACF208E
:1011F9007E0343DA20307E0343DA10C2D8C2717805
:10120900A2E67008D274E52F54E0F52FC27575294E
:10121900001205FE307409C3E529940A4002D2750B
:101229001205EF78023074027800C3E55C9840F04B
:10123900C2AF120613120613120613D2AF12060317
:10124900754C007888E6B40302612A1205EF788CA0
:10125900E6C39401500302132AE530C394015003F5
:1012690002132A207435C3E55C94FF500302132A44
:10127900C2AF120628D2AF1205FEC3E55C94015035
:10128900EFC2AF1206131205F4120613D2AF1205FC
:10129900FEC3E55C94FF40E902179B7F05D27F11ED
:1012A9002C1205FEC2AFC27F112CAE5CC3E55C9463
:1012B9007FD2AF40761205EAC2AF120628D2AFDF5D
:1012C900DC1163C3EE94057897F612060312163FF4
:1012D90012171E7F0AD27F112C1205FEC2AFC27FE0
:1012E900112CAE5CC3E55C947FD2AF50E61205EADF
:1012F900C2AF1206131205F4120613D2AFDFD611CC
:1013090063EE24037896F612060312163F12174D60
:101319001205FE112CC3E55C94FF5002416C0217C3
:101329009BC3E55C954C4003855C4C1205FE780136
:101339007988E7B403027805C3E55C984002414C1B
:10134900C2AF120628120628120628D2AF120603C7
:10135900753000E4F531F5320531E531F4703F05BA
:1013690032789AE67819146012783214600D787D13
:1013790014600878FA146003753200C3E5329840A6
:101389001D120F231205EA153275310078998673FB
:10139900C2AF120628D2AF789886731205FE1205DD
:1013A900F4E52A7005307402214778012074027827
:1013B90006C3E55C9840A17888E6C39403600312EC
:1013C90005FEE52A7003021147C2AF120F23E4F5A7
:1013D90022F523F524F525F526F567D2AF7885E6BC
:1013E900C333F565E4F544F545F546F547F548F5A4
:1013F90070F52CF52DF53775700875BB101205EAD7
:101409001208B8E5E820ECFBA8BDA9BEE97001F80F
:1014190088711208BC75700875BB10120FA4C2AF91
:101429007561FF120934852261852262852263D2A2
:10143900AF7522017524017525017526018560693D
:10144900756A0175B69075A903757A017888E6B44D
:101459000307C27D307602D27DD268D26975330026
:0F146900120E7D120EAC12095412095B120954B7
:1014780012095B120954120BE4120703120CE7124B
:101488000D3112095B120BD3306E0312070420676B
:101498000312085730670312089E120CE7120D60FA
:1014A80012095B120BE4306E03120740120CE712AC
:1014B8000DD712095B120BD3306E0312079E120C64
:1014C800E7120E0612095B120BE4306E031207FBDB
:1014D800120CE7120E7D12095B1208B8120BD31218
:1014E8000CE7120EAC1208BC12095B30692F856438
:1014F80061856462856069756A0179187A0CC3E54B
:101508003399400CC269D26A8A357561FF02152584
:10151800C3E55C9401400302147E0215AB306A1DDA
:10152800206C1AE535147006C26AD26B817EF535D7
:10153800C3E55C9401400302147E0215AB753600C6
:10154800788279A4E760027803C3E55F9850543045
:101558007404E52A604D7888E6B40317207D0520D9
:101568007607A17B307602A17B206C07D26C85645C
:101578006181BD78F0306C058564617820C3E541F0
:10158800985002817E306C1BC26CC27D307602D2CC
:101598007DD26A753512856461817E0536E55C60A9
:1015A80002A1AE753600C2AF120F237887E6FE7629
:1015B80002120FA47887EEF6E4F522F523F524F558
:1015C80025F526F565752C00752D0075A90075B6ED
:1015D80080757A00D2AF1205FE120F2378A4E66058
:1015E80006D293D295D297307409C3E53694044055
:1015F800022147615C901A0D7820121681E520B40B
:101608005A0CA3121681E520B4A50302161F120F67
:101618003812163F02163E901A0378807B0A12167B
:1016280081A308DBF9901A0F788C7B19121681A315
:1016380008DBF9901A2822C2AF1216C012169A9027
:101648001A00740E121686A37406121686A3741551
:10165800121686901A0378807B0A121685A308DB77
:10166800F9901A0F788C7B19121685A308DBF912EA
:1016780016D31216B1901A2822E493F622E6438F65
:1016880001538FFD75EF0275B7A575B7F1F0538F4C
:10169800FE22438F02438F0175EF0275B7A575B718
:1016A800F1901A0DF0538FFC22901A0D745AD186BE
:1016B800901A0E74A5D186227A3079D07820901AA3
:1016C80040D181E520F709A3DAF7227A3079D09062
:1016D8001A40E7D18609A3DAF922AB74A875BB01D1
:1016E800027984BB02027985BB03027986BB0402B6
:1016F8007992BB05027987BB060279A3BB070279F9
:101708009CBB08027988BB09027989E8F7227C0525
:10171800120603DCFB22C2AF12061312061A1206C7
:10172800211206281205F412061312061A120621AF
:101738001206281205F412061312061A12062112AE
:101748000628D2AF22C2AF12062812062112061AA4
:101758001206131205F412062812062112061A128E
:1017680006131205F412062812062112061A12068A
:1017780013D2AF22AE74AF75C2AF1206131206139E
:101788001206131205F4DEF21206281205F4DFF829
:10179800D2AF22F11EF116F1167574017575017537
:1017A8007600F17C7C05AD5C120603C3ED955C7098
:1017B800F5C3E55C9401400AC3E55C94FF4032023E
:1017C80017D7D1E2D13FF11EC2AF75EF12F116DC87
:1017D800D50576C3E5769403500280C6F1160575E3
:1017E800E5741490009F93F808C3E575985002803B
:1017F800AEF116F1160574C3E574940A5002809C84
:0E180800120F3812163FC2AF75EF12121716EC
:0319FD0002108E47
:101A00000E0615FFFFFFFF03040A0301015AA5019B
:101A1000FFFFFFFFFF03FFFFFF25D0FAFA04FF01DE
:091A2000007AFF0101000300FF40
:101A400023475F556C74726132304123202020207F
:101A500023424C48454C492346333930232020202B
:101A60002020202020202020202020202020202076
:101C0000C2AFC2D353D9BF7581C043B20343FF8073
:101C1000752438752503B1C975EF0275E24043F1AB
:101C20002053A4DF75D4FFD2857DFA780379E67C52
:101C300010752200752300901DD67B0675249875BB
:101C400025013085028142208508D8FBD9F9DCF7CF
:101C500081B4308508D8FBD9F9DCF781B4B189E4C7
:101C600093A3C39A6004DDC381B4DBDBB17B600264
:101C7000812B7B08E493FAA3B15CDBF87A30B15C8A
:101C8000752200752300B17BEAFCEBFDC3ED94FEE9
:101C9000400EB17B8A278B28ED30E0048A828B834B
:101CA000B17B7AC270D8C3ED94FE601350CEBD00F4
:101CB00025EC60097520007521FF0200008100A855
:101CC00027A9280809D804D90281D3B17FEA89AAB3
:101CD000F281C50D81A0C3ED94035049EDA2E092BD
:101CE000007AC5C3E5829400E583941C50902000DF
:101CF00010438F02438F0175B7A575B7F1F030001F
:101D00001FA827A9280809438F01538FFDD804D99C
:101D100002A12089AAE275B7A575B7F1F0A3A10DBC
:101D2000538FFC817C7AC1BD030CE493A3FAB140CC
:101D3000DCF8B138817C817EAA22AB23B15CEBFA5E
:101D4000EA6222752608C3E52313F523E52213F57D
:101D50002250066323A0632201D526EAB1C9B1C986
:101D600075260AEAF4200102D285300102C285B14B
:101D7000C9C3134002C201D526EB22B17FEAFB2082
:101D80008502A17F308502A184752608AE24AF2587
:101D9000C3EF13FFEE13FEB1CDB1C9C3EA13308513
:101DA000024480FA30E703632201C3E52313F523DD
:101DB000E52213F52250066323A0632201D526D91C
:101DC000E52265236523F52222AE24AF250E0FDE22
:101DD000FEDFFCD20122424C48656C693437316326
:041DE000F390060175
:00000001FF
